:02000000462890
:100008000800A301A200FF30A207031CA307031CDA
:1000180041280330A100E73013200728A101FC3E46
:10002800A000A109031C1E28FF300000A007031828
:100038001928A0076400A10F18280800A301A2002E
:1000480001302A28A101A301A2000530A800230835
:100058002102031D31282208200204300318013030
:10006800031902302805031DFF3041280038031DFD
:10007800FF300405031DFF30412883130313831247
:1000880064000800831607309F00990183129801C5
:100098008316023098008312D201CC010130D100BE
:1000A800C4011030C5002830C200C301C801C9010D
:1000B8002830C600C701831606108610061188016D
:1000C80087100710071187120512851283128801FD
:1000D8008614061587140715871607148512061047
:1000E8000130A300F4308A010620071001308A018C
:1000F800052007148A110A124D298A110A12AB2009
:1001080054088800071106158710861002308A01E6
:100118001220861487148A110A12AB205508880009
:10012800071106158710861002308A0112208614DE
:1001380087148A110A12AB20530888000615871005
:10014800861002308A01122086148714080087144A
:100158008316FF308800831207158614871006114E
:1001680002308A011220003008180130A000013046
:100178008A012620B200003088180130A000013022
:100188008A012620B4003208840034088A013A2003
:100198008A110A12031DAB280615871483168801D5
:1001A800831208004A08D5004B08D4002430D30035
:1001B8008A0181205608BE00BF013E08A0003F0802
:1001C800A10057088A0122208A110A12031DFD285E
:1001D8004E08D500C030D3008A018F205108BE07D1
:1001E8008A110A12031CE128BE0A8A110A12031D89
:1001F800E12808004A08D5004B08D4002430D30071
:100208008A01812008004E08D500C030D3008A0139
:100218008F200800CD01CC01640008304C028A11FF
:100228000A1203184C2920304D07C0001830031853
:10023800013EC10047304D07B60018300318013E93
:10024800B7004008A0004108A1003708A3003608FD
:100258008A0123208A110A12031D45294108CA0070
:100268004008CB008A01FE208A0107210230C0071E
:100278008A110A12031C1E29C10A8A110A12031DB7
:100288001E292830CD07CC0A8A110A12031D10290D
:1002980008004508D5004408D4004230D3008A013C
:1002A80081204308D5004208D4004330D3008A0196
:1002B80081204908D5004808D4004030D3008A017D
:1002C80081204708D5004608D4004130D3008A0170
:1002D80081208030D3008A019D20D501D4012430AB
:1002E800D3008A0181209830D3008A019D200130F3
:1002F800CC006400F1304C028A110A1203189C29C0
:100308000130CD00640041304D028A110A120318F1
:100318009729D501C030D3008A018F20CD0A8A11D0
:100328000A12031D8629CC0A8A110A12031D7D2987
:100338001030D500D4012430D3008A018120C001B7
:100348001030C1004008A0004108A1001430A300EB
:10035800D8308A0123208A110A12031DCA294108AC
:10036800CA004008CB00E030CE000130D600013092
:10037800D7008A01D6202830C0078A110A12031C28
:10038800A629C10A8A110A12031DA6292730C0000E
:100398001030C1004008A0004108A1001530A3009A
:1003A80028308A0123208A110A12031DF2294108E4
:1003B800CA004008CB00C130CE000130D600013061
:1003C800D7008A01D6202830C0078A110A12031CD8
:1003D800CE29C10A8A110A12031DCE29FF30CE0088
:1003E8000130D6002830D7000130D1001030CA00C3
:1003F800CB018A01D6201530CA00CB018A01D6204C
:100408001930CA00D830CB008A01D6209430D300E6
:100418008A019D20D5012930D4002430D3008A01D7
:100428008120CC01640024304C028A110A1203187E
:100438005D2A4C08233C8A110A12031C522A8A118D
:100448000A122A22D5008A110A12522A02308A0078
:100458004C08820754344F345334483449344234B6
:100468004134203454343634393436343334203437
:1004780043346F346E34743472346F346C346C3487
:1004880065347234203426342034533448344134AB
:100498005234503420344C34433444342030D50260
:1004A800C030D3008A018F20CC0A8A110A12031D9A
:1004B800162AD5015430D4002430D3008A01812073
:1004C800CC01640008304C028A110A120318902AE1
:1004D8004C08073C8A110A12031C852A8A110A1241
:1004E8007922D5008A110A12852A02308A004C081E
:1004F800820743346F3475346E347434653472341F
:100508003A342030D502C030D3008A018F20CC0A7B
:100518008A110A12031D652AD5016530D4002430DA
:10052800D3008A018120CC01640007304C028A1173
:100538000A120318C22A4C08063C8A110A12031C24
:10054800B72A8A110A12AC22D5008A110A12B72AD0
:1005580002308A004C08820742347534743474348B
:100568006F346E343A342030D502C030D3008A015B
:100578008F20CC0A8A110A12031D982AD501CA3085
:10058800D4002430D3008A018120CC0164002230B9
:100598004C028A110A1203182E2B4C08213C8A118E
:1005A8000A12031C232B8A110A12DE22D5008A1193
:0C05B8000A12232B03308A004C08002B91
:100600008207423479342034523461346E346A348F
:10061000693474342034443469346F346C34203495
:100620007534733469346E3467342034503449344B
:1006300043342034423461347334693463342034B5
:10064000503472346F342030D502C030D3008A0168
:100650008F20CC0A8A110A12031DCA2A9C30D300AB
:100660008A019D20D201D001F830CF004F08CE0082
:100670008A010E21D5016D30D4002430D3008A01C7
:10068000812064008A110A12061C702BCC016400C0
:1006900003304C028A110A1203186D2B4C08023CDD
:1006A0008A110A12031C622B8A110A125B23D500DD
:1006B0008A110A12622B03308A004C0882074F34D9
:1006C000463446342030D502C030D3008A018F2012
:1006D000CC0A8A110A12031D472B8A110A12972B82
:1006E000CC01640003304C028A110A120318972BC4
:1006F0004C08023C8A110A12031C8C2B8A110A1224
:100700008523D5008A110A128C2B03308A004C08ED
:1007100082074F344E3420342030D502C030D3000D
:100720008A018F20CC0A8A110A12031D712BC8304E
:100730008A010520CF0A8A110A12031D362B640094
:100740000A3052028A110A12031CA72BD201D501CA
:100750005D30D4002430D3008A0181205208093C46
:100760008A110A12031CC92B8A110A12BB23D50055
:100770008A110A12C92B03308A00520882073034CA
:100780003134323433343434353436343734383425
:1007900039342030D502C030D3008A018F20D20AEC
:1007A00064005008003C8A110A120319E02B14302F
:1007B000CA005008CB008A01FE20CE018A01072121
:1007C0001430CA003B305207CB004B08D0008A01DE
:1007D000FE20FF30CE008A0107218A01342B6300FE
:0407E0008A01EF2B70
:02400E00753DFE
:00000001FF
